:03000000020A866B
:0C0A8600787FE4F6D8FD758172020ACD7D
:10061A000A25642C2564452D342C2564452D340087
:10062A00656E74657220696E74657276616C287382
:10063A00293D0070726573732045534320746F20FF
:10064A0065786974000A0025642C2564452D342CCC
:10065A002564452D342C007E306D79335B5F707FC5
:10066A007B0A0D4475616C204368616E6E656C206F
:10067A004469676974616C20566F6C744D65746562
:10068A00722056312E3120283F2068656C7029006F
:10069A000A0D3E000A0D206120207072696E7420D6
:1006AA0072656164696E6773206175746F6D6174D8
:1006BA006963616C6C792020202020202020202072
:1006CA00202020202020202020200A0D2069202000
:1006DA0073657420696E74657276616C2873290972
:1006EA00090909090A0D205350206869742073709A
:1006FA006163652062617220746F20726561642093
:10070A0077697468206D616E75616C20656E7472AC
:02071A00790064
:100E3F00022A0005023B00050120000121000228C3
:100E4F000000042C000000000138610224000002A1
:070E5F004000010226000122
:080D41008F618E608D5F8C5EF6
:100D4900C295C297E4FBE55E548024FF9296D29740
:100D5900C297AF61AE60AD5FAC5E780112075B8F81
:0F0D6900618E608D5F8C5E0BBB20DBD295C295D7
:010D78002258
:100D79007F017E0A7D017C0A120D417F077E0B7D72
:100D8900077C0B120D417F007E097D007C09120D45
:100D9900417F007E0F7D007C0F120D417F017E0C8B
:070DA9007D017C0C020D41ED
:10037200E4F52FF52EF52DF52CE52F454EF52FE55D
:100382002EF52EE52DF52DE52CF52CAF2FAE2EAD4D
:100392002DFC781012075B8F2F8E2E8D2D8C2CE565
:1003A2002F4556F52FE52EF52EE52DF52DE52CF5ED
:1003B2002CE52FFFE52E4401FEE52DFDE52C440141
:1003C200FC120D41E4F52FF52EF52DF52CE52F4508
:1003D2004FF52FE52EF52EE52DF52DE52CF52CAF5D
:1003E2002FAE2EAD2DFC781012075B8F2F8E2E8D27
:1003F2002D8C2CE52F4557F52FE52EF52EE52DF505
:100402002DE52CF52CE52FFFE52E4402FEE52DFD12
:10041200E52C4402FC120D41E4F52FF52EF52DF5E5
:100422002CE52F4550F52FE52EF52EE52DF52DE582
:100432002CF52CAF2FAE2EAD2DFC781012075B8F52
:100442002F8E2E8D2D8C2CE52F4558F52FE52EF570
:100452002EE52DF52DE52CF52CE52FFFE52E440399
:10046200FEE52DFDE52C4403FC120D41E4F52FF5CC
:100472002EF52DF52CE5514480FFE52F4FF52FE5A4
:100482002EF52EE52DF52DE52CF52CAF2FAE2EAD4C
:100492002DFC781012075B8F2F8E2E8D2D8C2CE564
:1004A200594480FFE52F4FF52FE52EF52EE52DF56A
:1004B2002DE52CF52CE52FFFE52E4404FEE52DFD60
:1004C200E52C4404FC120D41E4F52FF52EF52DF533
:1004D2002CE52F4552F52FE52EF52EE52DF52DE5D0
:1004E2002CF52CAF2FAE2EAD2DFC781012075B8FA2
:1004F2002F8E2E8D2D8C2CE52F455AF52FE52EF5BE
:100502002EE52DF52DE52CF52CE52FFFE52E4405E6
:10051200FEE52DFDE52C4405FC120D41E4F52FF519
:100522002EF52DF52CE52F4553F52FE52EF52EE56D
:100532002DF52DE52CF52CAF2FAE2EAD2DFC781020
:1005420012075B8F2F8E2E8D2D8C2CE52F455BF5A0
:100552002FE52EF52EE52DF52DE52CF52CE52FFFBB
:10056200E52E4406FEE52DFDE52C4406FC120D4168
:10057200E4F52FF52EF52DF52CE52F4554F52FE555
:100582002EF52EE52DF52DE52CF52CAF2FAE2EAD4B
:100592002DFC781012075B8F2F8E2E8D2D8C2CE563
:1005A2002F455CF52FE52EF52EE52DF52DE52CF5E5
:1005B2002CE52FFFE52E4407FEE52DFDE52C440733
:1005C200FC120D41E4F52FF52EF52DF52CE52F4506
:1005D20055F52FE52EF52EE52DF52DE52CF52CAF55
:1005E2002FAE2EAD2DFC781012075B8F2F8E2E8D25
:1005F2002D8C2CE52F455DF52FE52EF52EE52DF5FD
:100602002DE52CF52CE52FFFE52E4408FEE52DFD0A
:08061200E52C4408FC020D4137
:03000B00020CBC28
:100CBC00C0E0C0D075D018438CDC053AE53A700220
:100CCC000539D39464E539648094804024753900E7
:100CDC00753A000525E525700205249541E540642B
:100CEC0080F8E5246480984008752400752500D2AE
:060CFC0007D0D0D0E03269
:03000300020B12DB
:100B1200C0E0C083C082C0D075D008308406752A78
:100B220000752B05E580540FFFAE2B74422EF8A6FC
:100B32000F74422EF8E6FF3395E0FE74612FF582C2
:100B420074063EF583E493FFC37408952B244EF894
:100B5200A60FE52B152B7002152AE52B452A7002EC
:100B6200D200E58030E504D2038002C203E5803082
:100B7200E604D2048002C204D0D0D082D083D0E076
:010B82003240
:03001300020B835A
:100B8300C0E0C083C082C0D075D01030A406753BCE
:100B930000753C05E5A0540FFFAE3C74302EF8A65B
:100BA3001774302EF8E6FF3395E0FE74612FF5825B
:100BB30074063EF583E493FFC37410953C244EF80A
:100BC300A617E53C153C7002153BE53C453B70021E
:100BD300D201E5A030E504D2058002C205E5A030CC
:100BE300E604D2068002C206D0D0D082D083D0E001
:010BF30032CF
:0E0F190075517E75520EE4F553F554F55522D0
:0E0F270075597E755A0EE4F55BF55CF55D229A
:10089F00200003020942E4F528F529AF47EF33950D
:1008AF00E0FE7C277D101207498E288F29AF46EF77
:1008BF003395E0FE7C037DE8120749EF2529F529E2
:1008CF00EE3528F528AF45EF3395E0FE7C007D64CB
:1008DF00120749EF2529F529EE3528F528AF44EF02
:1008EF003395E0FE7D0A120749EF2529F529EE35EC
:1008FF0028F528AF43EF3395E0FEEF2529F529EED4
:10090F003528F5282003057550018003E4F5504381
:10091F005180300403120F1912037220030FAE28F7
:10092F00AF297CFF7DFF1207498E288F2985284A22
:04093F0085294B2299
:100943002001030209E6E4F528F529AF35EF3395D5
:10095300E0FE7C277D101207498E288F29AF34EFE4
:100963003395E0FE7C037DE8120749EF2529F5293D
:10097300EE3528F528AF33EF3395E0FE7C007D6438
:10098300120749EF2529F529EE3528F528AF32EF6F
:100993003395E0FE7D0A120749EF2529F529EE3547
:1009A30028F528AF31EF3395E0FEEF2529F529EE41
:1009B3003528F5282005057558018003E4F55843CB
:1009C3005980300603120F2712037220050FAE2839
:1009D300AF297CFF7DFF1207498E288F2985284C7C
:0409E30085294D22F3
:0E0EFB00E4FFFE0FBF00010EBE75F8BF30F51C
:010F090022C5
:100E1500E4F53EF53F744E253FF876FF053FE53F87
:100E25007002053E6410453E70EB120372120EFB14
:0A0E3500E4F54EF54FF556F557228F
:100DB00030003230012F30022C300729C200C2012E
:100DC000C2077BFF7A06791A0527E5278526617019
:100DD00002052614F562854C63854D64854A658558
:060DE0004B6612007822B0
:080F60003098FDC298AF992200
:060DE6007BFF7A06796B29
:060DEC008B5E8A5F896046
:100DF200E4F561AB5EAA5FA960AF610561EF33956F
:100E0200E08F82F58312071CF5626006FF120E67FF
:020E120080E17D
:010E140022BB
:090F57007BFF7A06799A020DEC89
:0D0F3500309806120F608F3D22753DFF229F
:0B0F4200E53DB41B05C202120F572250
:100ED800E53DB43F0C7BFF7A06799E120DEC120FAC
:020EE80057228F
:100D0200E53D64697038C2AF7BFF7A06792A120D1D
:100D1200EC7B007A00794E7D107C001209E77B00A3
:100D22007A00794E1207F18E408F41900663E49368
:0F0D3200F54E900662E493F556E4F54FD2AF22EA
:100EAE00E53DB40D1120020E120DE6120F577526F8
:070EBE0000752701C20822A4
:100E8E00E53DB4611A7BFF7A06793D120DECD20274
:100E9E00752600752701E4F539F53AF524F5252276
:100C5900E53D6420705C200259300056300153C2D2
:100C690000C20120080B7BFF7A06794F120DECD2E6
:100C7900087BFF7A0679510527E5278526617002E9
:100C8900052614F562854C63854D64854A65854B57
:100C9900661200787B007A00794E7D107C0012097B
:100CA900E7900663E493F54E900662E493F556E403
:030CB900F54F22D2
:100BF400759850758921758DFDD28ED299D28CE469
:100C0400F5C843C902D2CA75CBFF75CAEAD288D2E5
:100C14008AD2A8D2AAD2A9D2AFD291120D79120D3A
:100C2400E6120F57120E15900663E493F54E9006E4
:100C340062E493F556120F35120F42120ED8120EBB
:100C4400AE120D02120E8E120C5912089F12094395
:050C5400120DB080E06C
:100A9200020BF4E493A3F8E493A34003F68001F27B
:100AA20008DFF48029E493A3F85407240CC8C33365
:100AB200C4540F4420C8834004F456800146F6DF34
:100AC200E4800B0102040810204080900E3FE47E77
:100AD200019360BCA3FF543F30E509541FFEE49329
:100AE200A360010ECF54C025E060A840B8E493A3F0
:100AF200FAE493A3F8E493A3C8C582C8CAC583CA1B
:100B0200F0A3C8C582C8CAC583CADFE9DEE780BED2
:010E6600008B
:10071C00BB010CE58229F582E5833AF583E0225092
:10072C0006E92582F8E622BBFE06E92582F8E222DC
:0D073C00E58229F582E5833AF583E49322F6
:10074900EF8DF0A4A8F0CF8CF0A428CE8DF0A42EC4
:02075900FE227E
:10075B00E8600FEFC333FFEE33FEED33FDEC33FCFC
:03076B00D8F122A0
:100E6700EFB40A07740D120E72740A309811A8991C
:100E7700B8130CC2983098FDA899C298B811F630EB
:070E870099FDC299F59922C3
:10001600E56D2461F8E6056D22785E301702786199
:10002600E475F0011207BB02076E2010EB7F2ED29B
:10003600108018EF540F2490D43440D4FF30140BA2
:10004600EF24BFB41A0050032461FFE56E60021569
:100056006E0571E5717002057030170D785EE475F6
:10006600F0011207BBEF020787020E677403D2176F
:100076008003E4C217F56D8B5E8A5F8960E4F56ED6
:10008600F570F571E56E60077F2012005180F575F9
:100096006FFFC211C210C212C213C215C216C21815
:1000A60012001FFF700D3017057F00120062AF713E
:1000B600AE7022B4255FC2D5C21412001FFF24D031
:1000C600B40A00501A75F00A786E30D50508B6FFE6
:1000D6000106C6A426F620D5047002D21380D924C0
:1000E600CFB41A00EF5004C2E5D214020262D21154
:1000F60080C6D21080C0D21280BCD2D580BAD215AA
:1001060080B47F201200512012077401B56E0040A2
:10011600F1120016FF12005102008AD218D2168080
:1001260095120016FB120016FA120016F94A4B70C9
:100136000679337A037BFF20122EE56E602A7E0055
:100146008E8275830012071C60060EEE656F70F0D6
:10015600C2D5EBC0E0EAC0E0E9C0E0EE1202A9D0E9
:10016600E0F9D0E0FAD0E0FB12076EFF60AAEBC020
:10017600E0EAC0E0E9C0E0120051D0E02401F9D085
:10018600E03400FAD0E0FBE56F0460DCD56FD9807F
:10019600877BFF7A0279A5D212809C79108002793A
:1001A60008C216C2188008D2D5790A8004790AC214
:1001B600D5E56F047002F56FE4FAFDFEFF12001636
:1001C600FC7B08201113120016FD7B1030100A125A
:1001D6000016FE120016FF7B20EC3382D592D55016
:1001E60013C3E43010069FFFE49EFEE42011039D36
:1001F600FDE49CFCE4CBF8C211EC700CCFCECDCC68
:10020600E824F8F870F38017C3EF33FFEE33FEED02
:1002160033FDEC33FCEB33FB994002FB0FD8E9EBE3
:10022600301105F8D0E0C448B211C0E00AEC4D4EDA
:100236004F78207B0070C2EAB56F0040BCC0E01268
:1002460002ABD0F0D0E0201104C4C0E0C4B211C0AB
:10025600F012003AD0F0D5F0EB02008A1207CB017B
:10026600275301A15800F84C00F44201A54F01ADF7
:0F0276004401AD49010D4301B35501974601976E
:100285004501974703535000FC2D01002E01232BF8
:10029500010423012120033C2A00BC480000011B66
:1002A5003F3F3F00790AA2D5201314301509B91034
:1002B500020404B9080104A2D52016025001042045
:1002C50012689212B56E005034C0E07F20301319C9
:1002D5007F30A21272167215500F120302C212C29B
:1002E50016C215C2187F30800F301503E9C0E01221
:1002F5000051301503D0E0F9D0E0B56ECC301517BC
:100305007F30B9100C1200517F583014077F788068
:1003150003B908031200513012057F2D0200517FE9
:10032500202018F87F2B2016F322921280CF286EFA
:10033500756C6C2900D2111200163011F8C21178B3
:100345006E30D50108F60200BC2D50434958120005
:10035500162403B405004001E490034E93120042B5
:0D036500743A120042D213756E040201A119
:1009E7008B5E8A5F89608C618D62E4F563F564E5EF
:1009F7006224FFFFE56134FFFEC3E5649FEE648078
:100A0700F8E5636480985066120EEAAB5EAA5FA9A8
:100A170060856482856383EF120799640A604FAB30
:100A27005EAA5FA96085648285638312071CB40888
:100A37001AE56445636008E5641564700215637F11
:100A470020120E677F08120E6780A4AB5EAA5FA90B
:100A57006085648285638312071CFF64116090EFD1
:100A67006413608B0564E564708505638081AB5E04
:0F0A7700AA5FA960856482856383E412079922D0
:1007F1008B5E8A5F8960AB5EAA5FA96012076EFF9C
:10080100120EC5500D74012560F560E4355FF55F8A
:1008110080E4D210AB5EAA5FA96012076EFF642B61
:100821006004EFB42D1BAB5E0560E560AA5F70024A
:10083100055F14F912076E642D6003D38001C39222
:1008410010E4F561F562AB5EAA5FA96012076EFF65
:10085100120F0A5036AB5EAA5FA96012076EFF3312
:1008610095E0FEEF24D0FBEE34FFFAAE61AF627C7F
:10087100007D0A120749EF2BF562EE3AF56174012A
:100881002560F560E4355FF55F80BB301006AE6131
:0E089100AF628009C3E49562FFE49561FE2228
:10076E00BB010689828A83E0225002E722BBFE0289
:09077E00E32289828A83E49322BC
:10078700BB010689828A83F0225002F722BBFE0151
:02079700F3224B
:10079900F8BB010DE58229F582E5833AF583E8F096
:1007A900225006E92582C8F622BBFE05E92582C842
:0207B900F2222A
:1007BB00FAE6FB0808E6F925F0F618E6CA3AF6223F
:1007CB00D083D082F8E4937012740193700DA3A3BD
:1007DB0093F8740193F5828883E4737402936860D1
:0607EB00EFA3A3A380DFD1
:100EEA0010190B120F4DBF0D027F0A020E67AF7267
:010EFA0022D5
:0F0F0A00EFC394304007EF943A50028001C322A6
:100EC500EFC394094005EF940E4003BF2003D38080
:030ED50001C32234
:0A0F4D003098FDAF99C2987E002293
:00000001FF
